:0A00060000308A00352800002B307E
:100010008400000803191B280130F800F701F70BD2
:100020000F28F80B0E284A30F700F70B15280000B0
:100030000000800B0C288A112E28A901A80129088C
:100040002702031C3428031D292826082802031828
:1000500034280430AA00FA30AB000728AA0B2B285A
:10006000A80A0319A90A1F28003484011F30830538
:1000700083161F08C0399F009B01073083129F0021
:10008000A1010230A000A301A200A501A4008316D3
:100090008501FF3086008312850183168113831248
:1000A00005142108A7002008A6001D2005108514AE
:1000B0002308A7002208A6001D2085100515250885
:1000C000A7002408A6001D20051183164F286300F1
:040000008A01032846
:02400E00693F08
:00000001FF
